 management_ext

 Timestamp is 6f047f5c (reproducible build file hash)

 Preferred load address is 0000000180000000

 Start         Length     Name                   Class
 0001:00000000 00002ee0H .text$mn                CODE
 0001:00002ee0 00000036H .text$mn$00             CODE
 0001:00002f16 00000092H .text$x                 CODE
 0002:00000000 00000220H .idata$5                DATA
 0002:00000220 00000038H .00cfg                  DATA
 0002:00000258 00000008H .CRT$XCA                DATA
 0002:00000260 00000008H .CRT$XCZ                DATA
 0002:00000268 00000008H .CRT$XIA                DATA
 0002:00000270 00000008H .CRT$XIZ                DATA
 0002:00000278 00000008H .CRT$XPA                DATA
 0002:00000280 00000008H .CRT$XPZ                DATA
 0002:00000288 00000008H .CRT$XTA                DATA
 0002:00000290 00000010H .CRT$XTZ                DATA
 0002:00000298 00000000H .gehcont$y              DATA
 0002:00000298 00000000H .gfids$y                DATA
 0002:000002a0 00000960H .rdata                  DATA
 0002:00000c00 00000000H .rdata$CastGuardVftablesA DATA
 0002:00000c00 00000000H .rdata$CastGuardVftablesC DATA
 0002:00000c00 0000006cH .rdata$voltmd           DATA
 0002:00000c6c 000002bcH .rdata$zzzdbg           DATA
 0002:00000f28 00000008H .rtc$IAA                DATA
 0002:00000f30 00000008H .rtc$IZZ                DATA
 0002:00000f38 00000008H .rtc$TAA                DATA
 0002:00000f40 00000008H .rtc$TZZ                DATA
 0002:00000f48 00000318H .xdata                  DATA
 0002:00001260 0000082cH .edata                  DATA
 0002:00001a8c 000000dcH .idata$2                DATA
 0002:00001b68 00000018H .idata$3                DATA
 0002:00001b80 00000220H .idata$4                DATA
 0002:00001da0 0000058eH .idata$6                DATA
 0003:00000000 000000d0H .data                   DATA
 0003:000000d0 00000708H .bss                    DATA
 0004:00000000 00000354H .pdata                  DATA
 0005:00000000 00000060H .rsrc$01                DATA
 0005:00000060 00000330H .rsrc$02                DATA

  Address         Publics by Value              Rva+Base               Lib:Object

 0000:00000000       __AbsoluteZero             0000000000000000     <absolute>
 0000:00000000       ___safe_se_handler_count   0000000000000000     <absolute>
 0000:00000000       ___safe_se_handler_table   0000000000000000     <absolute>
 0000:00000000       __arm64x_extra_rfe_table   0000000000000000     <absolute>
 0000:00000000       __arm64x_extra_rfe_table_size 0000000000000000     <absolute>
 0000:00000000       __arm64x_native_entrypoint 0000000000000000     <absolute>
 0000:00000000       __arm64x_redirection_metadata 0000000000000000     <absolute>
 0000:00000000       __arm64x_redirection_metadata_count 0000000000000000     <absolute>
 0000:00000000       __dynamic_value_reloc_table 0000000000000000     <absolute>
 0000:00000000       __enclave_config           0000000000000000     <absolute>
 0000:00000000       __guard_check_icall_a64n_fptr 0000000000000000     <absolute>
 0000:00000000       __guard_eh_cont_count      0000000000000000     <absolute>
 0000:00000000       __guard_eh_cont_table      0000000000000000     <absolute>
 0000:00000000       __guard_fids_count         0000000000000000     <absolute>
 0000:00000000       __guard_fids_table         0000000000000000     <absolute>
 0000:00000000       __guard_iat_count          0000000000000000     <absolute>
 0000:00000000       __guard_iat_table          0000000000000000     <absolute>
 0000:00000000       __guard_longjmp_count      0000000000000000     <absolute>
 0000:00000000       __guard_longjmp_table      0000000000000000     <absolute>
 0000:00000000       __hybrid_auxiliary_delayload_iat 0000000000000000     <absolute>
 0000:00000000       __hybrid_auxiliary_delayload_iat_copy 0000000000000000     <absolute>
 0000:00000000       __hybrid_auxiliary_iat     0000000000000000     <absolute>
 0000:00000000       __hybrid_auxiliary_iat_copy 0000000000000000     <absolute>
 0000:00000000       __hybrid_code_map          0000000000000000     <absolute>
 0000:00000000       __hybrid_code_map_count    0000000000000000     <absolute>
 0000:00000000       __hybrid_image_info_bitfield 0000000000000000     <absolute>
 0000:00000000       __x64_code_ranges_to_entry_points 0000000000000000     <absolute>
 0000:00000000       __x64_code_ranges_to_entry_points_count 0000000000000000     <absolute>
 0000:00000100       __guard_flags              0000000000000100     <absolute>
 0000:00000000       __ImageBase                0000000180000000     <linker-defined>
 0001:00000000       Java_com_sun_management_internal_DiagnosticCommandImpl_executeDiagnosticCommand 0000000180001000 f   DiagnosticCommandImpl.obj
 0001:00000014       Java_com_sun_management_internal_DiagnosticCommandImpl_getDiagnosticCommandInfo 0000000180001014 f   DiagnosticCommandImpl.obj
 0001:000003f4       Java_com_sun_management_internal_DiagnosticCommandImpl_getDiagnosticCommands 00000001800013f4 f   DiagnosticCommandImpl.obj
 0001:00000404       Java_com_sun_management_internal_DiagnosticCommandImpl_setNotificationEnabled 0000000180001404 f   DiagnosticCommandImpl.obj
 0001:00000434       getDiagnosticCommandArgumentInfoArray 0000000180001434 f   DiagnosticCommandImpl.obj
 0001:00000724       Java_com_sun_management_internal_Flag_getAllFlagNames 0000000180001724 f   Flag.obj
 0001:00000734       Java_com_sun_management_internal_Flag_getFlags 0000000180001734 f   Flag.obj
 0001:000009b8       Java_com_sun_management_internal_Flag_getInternalFlagCount 00000001800019b8 f   Flag.obj
 0001:000009cc       Java_com_sun_management_internal_Flag_initialize 00000001800019cc f   Flag.obj
 0001:00000a88       Java_com_sun_management_internal_Flag_setBooleanValue 0000000180001a88 f   Flag.obj
 0001:00000aac       Java_com_sun_management_internal_Flag_setDoubleValue 0000000180001aac f   Flag.obj
 0001:00000ac8       Java_com_sun_management_internal_Flag_setLongValue 0000000180001ac8 f   Flag.obj
 0001:00000ac8       Java_com_sun_management_internal_Flag_setStringValue 0000000180001ac8 f   Flag.obj
 0001:00000b18       Java_com_sun_management_internal_GarbageCollectorExtImpl_setNotificationEnabled 0000000180001b18 f   GarbageCollectorExtImpl.obj
 0001:00000b58       Java_com_sun_management_internal_GcInfoBuilder_fillGcAttributeInfo 0000000180001b58 f   GcInfoBuilder.obj
 0001:00000d38       Java_com_sun_management_internal_GcInfoBuilder_getLastGcInfo0 0000000180001d38 f   GcInfoBuilder.obj
 0001:00001020       Java_com_sun_management_internal_GcInfoBuilder_getNumGcExtAttributes 0000000180002020 f   GcInfoBuilder.obj
 0001:00001058       Java_com_sun_management_internal_HotSpotDiagnostic_dumpHeap0 0000000180002058 f   HotSpotDiagnostic.obj
 0001:0000106c       Java_com_sun_management_internal_OperatingSystemImpl_getCommittedVirtualMemorySize0 000000018000206c f   OperatingSystemImpl.obj
 0001:000010c0       Java_com_sun_management_internal_OperatingSystemImpl_getFreePhysicalMemorySize0 00000001800020c0 f   OperatingSystemImpl.obj
 0001:00001100       Java_com_sun_management_internal_OperatingSystemImpl_getFreeSwapSpaceSize0 0000000180002100 f   OperatingSystemImpl.obj
 0001:00001140       Java_com_sun_management_internal_OperatingSystemImpl_getProcessCpuLoad0 0000000180002140 f   OperatingSystemImpl.obj
 0001:000011ac       Java_com_sun_management_internal_OperatingSystemImpl_getProcessCpuTime0 00000001800021ac f   OperatingSystemImpl.obj
 0001:00001200       Java_com_sun_management_internal_OperatingSystemImpl_getSystemCpuLoad0 0000000180002200 f   OperatingSystemImpl.obj
 0001:00001254       Java_com_sun_management_internal_OperatingSystemImpl_getTotalPhysicalMemorySize0 0000000180002254 f   OperatingSystemImpl.obj
 0001:00001294       Java_com_sun_management_internal_OperatingSystemImpl_getTotalSwapSpaceSize0 0000000180002294 f   OperatingSystemImpl.obj
 0001:000012d4       Java_com_sun_management_internal_OperatingSystemImpl_initialize0 00000001800022d4 f   OperatingSystemImpl.obj
 0001:00001308       __local_stdio_printf_options 0000000180002308 f i OperatingSystemImpl.obj
 0001:00001310       _snprintf                  0000000180002310 f i OperatingSystemImpl.obj
 0001:0000207c       JNI_OnLoad                 000000018000307c f   management_ext.obj
 0001:000020e3       JVM_GetManagement          00000001800030e3 f   jvm:jvm.dll
 0001:000020e9       GetProcessMemoryInfo       00000001800030e9 f   psapi:PSAPI.DLL
 0001:000020ef       JNU_ThrowByName            00000001800030ef f   java:java.dll
 0001:000020f5       JNU_ThrowNullPointerException 00000001800030f5 f   java:java.dll
 0001:000020fb       JNU_ThrowOutOfMemoryError  00000001800030fb f   java:java.dll
 0001:00002101       JNU_NewObjectByName        0000000180003101 f   java:java.dll
 0001:00002107       JNU_ThrowIllegalArgumentException 0000000180003107 f   java:java.dll
 0001:0000210d       JNU_ThrowInternalError     000000018000310d f   java:java.dll
 0001:00002113       JNU_GetStaticFieldByName   0000000180003113 f   java:java.dll
 0001:0000211c       __GSHandlerCheck           000000018000311c f   MSVCRT:gshandler.obj
 0001:0000213c       __GSHandlerCheckCommon     000000018000313c f   MSVCRT:gshandler.obj
 0001:000021b0       __security_check_cookie    00000001800031b0 f   MSVCRT:amdsecgs.obj
 0001:000024f0       _DllMainCRTStartup         00000001800034f0 f   MSVCRT:dll_dllmain.obj
 0001:00002530       __raise_securityfailure    0000000180003530 f   MSVCRT:gs_report.obj
 0001:00002564       __report_gsfailure         0000000180003564 f   MSVCRT:gs_report.obj
 0001:000026ac       __security_init_cookie     00000001800036ac f   MSVCRT:gs_support.obj
 0001:00002758       DllMain                    0000000180003758 f   MSVCRT:dll_dllmain_stub.obj
 0001:0000277c       ?__scrt_initialize_type_info@@YAXXZ 000000018000377c f   MSVCRT:tncleanup.obj
 0001:0000278c       ?__scrt_uninitialize_type_info@@YAXXZ 000000018000378c f   MSVCRT:tncleanup.obj
 0001:00002798       __local_stdio_scanf_options 0000000180003798 f i MSVCRT:default_local_stdio_options.obj
 0001:000027a0       __scrt_initialize_default_local_stdio_options 00000001800037a0 f   MSVCRT:default_local_stdio_options.obj
 0001:000027bc       __scrt_acquire_startup_lock 00000001800037bc f   MSVCRT:utility.obj
 0001:000027f8       __scrt_dllmain_after_initialize_c 00000001800037f8 f   MSVCRT:utility.obj
 0001:0000282c       __scrt_dllmain_before_initialize_c 000000018000382c f   MSVCRT:utility.obj
 0001:00002844       __scrt_dllmain_crt_thread_attach 0000000180003844 f   MSVCRT:utility.obj
 0001:0000286c       __scrt_dllmain_crt_thread_detach 000000018000386c f   MSVCRT:utility.obj
 0001:00002884       __scrt_dllmain_exception_filter 0000000180003884 f   MSVCRT:utility.obj
 0001:000028e4       __scrt_dllmain_uninitialize_c 00000001800038e4 f   MSVCRT:utility.obj
 0001:00002914       __scrt_dllmain_uninitialize_critical 0000000180003914 f   MSVCRT:utility.obj
 0001:00002928       __scrt_initialize_crt      0000000180003928 f   MSVCRT:utility.obj
 0001:00002974       __scrt_initialize_onexit_tables 0000000180003974 f   MSVCRT:utility.obj
 0001:00002a00       __scrt_is_nonwritable_in_current_image 0000000180003a00 f   MSVCRT:utility.obj
 0001:00002a98       __scrt_release_startup_lock 0000000180003a98 f   MSVCRT:utility.obj
 0001:00002abc       __scrt_uninitialize_crt    0000000180003abc f   MSVCRT:utility.obj
 0001:00002ae8       __scrt_get_dyn_tls_init_callback 0000000180003ae8 f   MSVCRT:dyn_tls_init.obj
 0001:00002af0       __crt_debugger_hook        0000000180003af0 f   MSVCRT:utility_desktop.obj
 0001:00002af8       __scrt_fastfail            0000000180003af8 f   MSVCRT:utility_desktop.obj
 0001:00002c44       _RTC_Initialize            0000000180003c44 f   MSVCRT:initsect.obj
 0001:00002c80       _RTC_Terminate             0000000180003c80 f   MSVCRT:initsect.obj
 0001:00002cbc       _guard_check_icall_nop     0000000180003cbc f i MSVCRT:guard_support.obj
 0001:00002cc0       __isa_available_init       0000000180003cc0 f   MSVCRT:cpu_disp.obj
 0001:00002e6c       _get_startup_argv_mode     0000000180003e6c f   MSVCRT:argv_mode.obj
 0001:00002e74       __scrt_is_ucrt_dll_in_use  0000000180003e74 f   MSVCRT:ucrt_detection.obj
 0001:00002e80       memset                     0000000180003e80 f   vcruntime:VCRUNTIME140.dll
 0001:00002e86       strrchr                    0000000180003e86 f   vcruntime:VCRUNTIME140.dll
 0001:00002e8c       __C_specific_handler       0000000180003e8c f   vcruntime:VCRUNTIME140.dll
 0001:00002e92       __std_type_info_destroy_list 0000000180003e92 f   vcruntime:VCRUNTIME140.dll
 0001:00002e98       strlen                     0000000180003e98 f   ucrt:api-ms-win-crt-string-l1-1-0.dll
 0001:00002e9e       _initterm                  0000000180003e9e f   ucrt:api-ms-win-crt-runtime-l1-1-0.dll
 0001:00002ea4       _initterm_e                0000000180003ea4 f   ucrt:api-ms-win-crt-runtime-l1-1-0.dll
 0001:00002eaa       _seh_filter_dll            0000000180003eaa f   ucrt:api-ms-win-crt-runtime-l1-1-0.dll
 0001:00002eb0       _configure_narrow_argv     0000000180003eb0 f   ucrt:api-ms-win-crt-runtime-l1-1-0.dll
 0001:00002eb6       _initialize_narrow_environment 0000000180003eb6 f   ucrt:api-ms-win-crt-runtime-l1-1-0.dll
 0001:00002ebc       _initialize_onexit_table   0000000180003ebc f   ucrt:api-ms-win-crt-runtime-l1-1-0.dll
 0001:00002ec2       _execute_onexit_table      0000000180003ec2 f   ucrt:api-ms-win-crt-runtime-l1-1-0.dll
 0001:00002ec8       _cexit                     0000000180003ec8 f   ucrt:api-ms-win-crt-runtime-l1-1-0.dll
 0001:00002ed0       __acrt_initialize          0000000180003ed0 f   MSVCRT:ucrt_stubs.obj
 0001:00002ed0       __acrt_thread_attach       0000000180003ed0 f   MSVCRT:ucrt_stubs.obj
 0001:00002ed0       __acrt_thread_detach       0000000180003ed0 f   MSVCRT:ucrt_stubs.obj
 0001:00002ed0       __acrt_uninitialize        0000000180003ed0 f   MSVCRT:ucrt_stubs.obj
 0001:00002ed0       __acrt_uninitialize_critical 0000000180003ed0 f   MSVCRT:ucrt_stubs.obj
 0001:00002ed0       __scrt_stub_for_acrt_initialize 0000000180003ed0 f   MSVCRT:ucrt_stubs.obj
 0001:00002ed0       __scrt_stub_for_acrt_thread_attach 0000000180003ed0 f   MSVCRT:ucrt_stubs.obj
 0001:00002ed0       __scrt_stub_for_acrt_thread_detach 0000000180003ed0 f   MSVCRT:ucrt_stubs.obj
 0001:00002ed0       __scrt_stub_for_acrt_uninitialize 0000000180003ed0 f   MSVCRT:ucrt_stubs.obj
 0001:00002ed0       __scrt_stub_for_acrt_uninitialize_critical 0000000180003ed0 f   MSVCRT:ucrt_stubs.obj
 0001:00002ed0       __vcrt_initialize          0000000180003ed0 f   MSVCRT:ucrt_stubs.obj
 0001:00002ed0       __vcrt_thread_attach       0000000180003ed0 f   MSVCRT:ucrt_stubs.obj
 0001:00002ed0       __vcrt_thread_detach       0000000180003ed0 f   MSVCRT:ucrt_stubs.obj
 0001:00002ed0       __vcrt_uninitialize        0000000180003ed0 f   MSVCRT:ucrt_stubs.obj
 0001:00002ed0       __vcrt_uninitialize_critical 0000000180003ed0 f   MSVCRT:ucrt_stubs.obj
 0001:00002ed4       __scrt_stub_for_is_c_termination_complete 0000000180003ed4 f   MSVCRT:ucrt_stubs.obj
 0001:00002ed4       _is_c_termination_complete 0000000180003ed4 f   MSVCRT:ucrt_stubs.obj
 0001:00002ed7       memcpy                     0000000180003ed7 f   vcruntime:VCRUNTIME140.dll
 0001:00002ef0       _guard_dispatch_icall_nop  0000000180003ef0 f   MSVCRT:guard_dispatch.obj
 0001:00002f10       _guard_xfg_dispatch_icall_nop 0000000180003f10 f   MSVCRT:guard_xfg_dispatch.obj
 0002:00000000       __imp_InitializeSListHead  0000000180004000     kernel32:KERNEL32.dll
 0002:00000008       __imp_DisableThreadLibraryCalls 0000000180004008     kernel32:KERNEL32.dll
 0002:00000010       __imp_GetSystemTimeAsFileTime 0000000180004010     kernel32:KERNEL32.dll
 0002:00000018       __imp_GetCurrentProcessId  0000000180004018     kernel32:KERNEL32.dll
 0002:00000020       __imp_QueryPerformanceCounter 0000000180004020     kernel32:KERNEL32.dll
 0002:00000028       __imp_IsProcessorFeaturePresent 0000000180004028     kernel32:KERNEL32.dll
 0002:00000030       __imp_TerminateProcess     0000000180004030     kernel32:KERNEL32.dll
 0002:00000038       __imp_SetUnhandledExceptionFilter 0000000180004038     kernel32:KERNEL32.dll
 0002:00000040       __imp_UnhandledExceptionFilter 0000000180004040     kernel32:KERNEL32.dll
 0002:00000048       __imp_RtlVirtualUnwind     0000000180004048     kernel32:KERNEL32.dll
 0002:00000050       __imp_GetLastError         0000000180004050     kernel32:KERNEL32.dll
 0002:00000058       __imp_InitializeCriticalSection 0000000180004058     kernel32:KERNEL32.dll
 0002:00000060       __imp_EnterCriticalSection 0000000180004060     kernel32:KERNEL32.dll
 0002:00000068       __imp_LeaveCriticalSection 0000000180004068     kernel32:KERNEL32.dll
 0002:00000070       __imp_GetProcessTimes      0000000180004070     kernel32:KERNEL32.dll
 0002:00000078       __imp_GetCurrentProcess    0000000180004078     kernel32:KERNEL32.dll
 0002:00000080       __imp_GetCurrentThreadId   0000000180004080     kernel32:KERNEL32.dll
 0002:00000088       __imp_GlobalMemoryStatusEx 0000000180004088     kernel32:KERNEL32.dll
 0002:00000090       __imp_GetSystemInfo        0000000180004090     kernel32:KERNEL32.dll
 0002:00000098       __imp_FreeLibrary          0000000180004098     kernel32:KERNEL32.dll
 0002:000000a0       __imp_GetModuleFileNameA   00000001800040a0     kernel32:KERNEL32.dll
 0002:000000a8       __imp_GetProcAddress       00000001800040a8     kernel32:KERNEL32.dll
 0002:000000b0       __imp_LoadLibraryA         00000001800040b0     kernel32:KERNEL32.dll
 0002:000000b8       __imp_RtlCaptureContext    00000001800040b8     kernel32:KERNEL32.dll
 0002:000000c0       __imp_RtlLookupFunctionEntry 00000001800040c0     kernel32:KERNEL32.dll
 0002:000000c8       __imp_IsDebuggerPresent    00000001800040c8     kernel32:KERNEL32.dll
 0002:000000d0       \177KERNEL32_NULL_THUNK_DATA 00000001800040d0     kernel32:KERNEL32.dll
 0002:000000d8       __imp_GetProcessMemoryInfo 00000001800040d8     psapi:PSAPI.DLL
 0002:000000e0       \177PSAPI_NULL_THUNK_DATA  00000001800040e0     psapi:PSAPI.DLL
 0002:000000e8       __imp___std_type_info_destroy_list 00000001800040e8     vcruntime:VCRUNTIME140.dll
 0002:000000f0       __imp_memset               00000001800040f0     vcruntime:VCRUNTIME140.dll
 0002:000000f8       __imp___C_specific_handler 00000001800040f8     vcruntime:VCRUNTIME140.dll
 0002:00000100       __imp_strrchr              0000000180004100     vcruntime:VCRUNTIME140.dll
 0002:00000108       __imp_memcpy               0000000180004108     vcruntime:VCRUNTIME140.dll
 0002:00000110       \177VCRUNTIME140_NULL_THUNK_DATA 0000000180004110     vcruntime:VCRUNTIME140.dll
 0002:00000118       __imp__itoa                0000000180004118     ucrt:api-ms-win-crt-convert-l1-1-0.dll
 0002:00000118       __imp_itoa                 0000000180004118     ucrt:api-ms-win-crt-convert-l1-1-0.dll
 0002:00000120       \177api-ms-win-crt-convert-l1-1-0_NULL_THUNK_DATA 0000000180004120     ucrt:api-ms-win-crt-convert-l1-1-0.dll
 0002:00000128       __imp_free                 0000000180004128     ucrt:api-ms-win-crt-heap-l1-1-0.dll
 0002:00000130       __imp_malloc               0000000180004130     ucrt:api-ms-win-crt-heap-l1-1-0.dll
 0002:00000138       __imp_calloc               0000000180004138     ucrt:api-ms-win-crt-heap-l1-1-0.dll
 0002:00000140       \177api-ms-win-crt-heap-l1-1-0_NULL_THUNK_DATA 0000000180004140     ucrt:api-ms-win-crt-heap-l1-1-0.dll
 0002:00000148       __imp__execute_onexit_table 0000000180004148     ucrt:api-ms-win-crt-runtime-l1-1-0.dll
 0002:00000150       __imp__cexit               0000000180004150     ucrt:api-ms-win-crt-runtime-l1-1-0.dll
 0002:00000158       __imp__initialize_onexit_table 0000000180004158     ucrt:api-ms-win-crt-runtime-l1-1-0.dll
 0002:00000160       __imp__initialize_narrow_environment 0000000180004160     ucrt:api-ms-win-crt-runtime-l1-1-0.dll
 0002:00000168       __imp__initterm            0000000180004168     ucrt:api-ms-win-crt-runtime-l1-1-0.dll
 0002:00000170       __imp__configure_narrow_argv 0000000180004170     ucrt:api-ms-win-crt-runtime-l1-1-0.dll
 0002:00000178       __imp__getpid              0000000180004178     ucrt:api-ms-win-crt-runtime-l1-1-0.dll
 0002:00000180       __imp__seh_filter_dll      0000000180004180     ucrt:api-ms-win-crt-runtime-l1-1-0.dll
 0002:00000188       __imp__initterm_e          0000000180004188     ucrt:api-ms-win-crt-runtime-l1-1-0.dll
 0002:00000190       \177api-ms-win-crt-runtime-l1-1-0_NULL_THUNK_DATA 0000000180004190     ucrt:api-ms-win-crt-runtime-l1-1-0.dll
 0002:00000198       __imp___stdio_common_vsprintf 0000000180004198     ucrt:api-ms-win-crt-stdio-l1-1-0.dll
 0002:000001a0       \177api-ms-win-crt-stdio-l1-1-0_NULL_THUNK_DATA 00000001800041a0     ucrt:api-ms-win-crt-stdio-l1-1-0.dll
 0002:000001a8       __imp_strlen               00000001800041a8     ucrt:api-ms-win-crt-string-l1-1-0.dll
 0002:000001b0       __imp_strncpy              00000001800041b0     ucrt:api-ms-win-crt-string-l1-1-0.dll
 0002:000001b8       \177api-ms-win-crt-string-l1-1-0_NULL_THUNK_DATA 00000001800041b8     ucrt:api-ms-win-crt-string-l1-1-0.dll
 0002:000001c0       __imp_clock                00000001800041c0     ucrt:api-ms-win-crt-time-l1-1-0.dll
 0002:000001c8       \177api-ms-win-crt-time-l1-1-0_NULL_THUNK_DATA 00000001800041c8     ucrt:api-ms-win-crt-time-l1-1-0.dll
 0002:000001d0       __imp_JNU_ThrowIllegalArgumentException 00000001800041d0     java:java.dll
 0002:000001d8       __imp_JNU_ThrowInternalError 00000001800041d8     java:java.dll
 0002:000001e0       __imp_JNU_GetStaticFieldByName 00000001800041e0     java:java.dll
 0002:000001e8       __imp_JNU_ThrowNullPointerException 00000001800041e8     java:java.dll
 0002:000001f0       __imp_JNU_ThrowByName      00000001800041f0     java:java.dll
 0002:000001f8       __imp_JNU_ThrowOutOfMemoryError 00000001800041f8     java:java.dll
 0002:00000200       __imp_JNU_NewObjectByName  0000000180004200     java:java.dll
 0002:00000208       \177java_NULL_THUNK_DATA   0000000180004208     java:java.dll
 0002:00000210       __imp_JVM_GetManagement    0000000180004210     jvm:jvm.dll
 0002:00000218       \177jvm_NULL_THUNK_DATA    0000000180004218     jvm:jvm.dll
 0002:00000220       __guard_check_icall_fptr   0000000180004220     MSVCRT:guard_support.obj
 0002:00000228       __guard_xfg_check_icall_fptr 0000000180004228     MSVCRT:guard_support.obj
 0002:00000230       __guard_dispatch_icall_fptr 0000000180004230     MSVCRT:guard_support.obj
 0002:00000238       __guard_xfg_dispatch_icall_fptr 0000000180004238     MSVCRT:guard_support.obj
 0002:00000240       __guard_xfg_table_dispatch_icall_fptr 0000000180004240     MSVCRT:guard_support.obj
 0002:00000248       __castguard_check_failure_os_handled_fptr 0000000180004248     MSVCRT:guard_support.obj
 0002:00000250       __guard_memcpy_fptr        0000000180004250     vcruntime:softmemtag.obj
 0002:00000258       __xc_a                     0000000180004258     MSVCRT:initializers.obj
 0002:00000260       __xc_z                     0000000180004260     MSVCRT:initializers.obj
 0002:00000268       __xi_a                     0000000180004268     MSVCRT:initializers.obj
 0002:00000270       __xi_z                     0000000180004270     MSVCRT:initializers.obj
 0002:00000278       __xp_a                     0000000180004278     MSVCRT:initializers.obj
 0002:00000280       __xp_z                     0000000180004280     MSVCRT:initializers.obj
 0002:00000288       __xt_a                     0000000180004288     MSVCRT:initializers.obj
 0002:00000290       __xt_z                     0000000180004290     MSVCRT:initializers.obj
 0002:000002a0       ??_C@_0FA@KDGODBFA@JMX?5interface?5to?5diagnostic?5fra@ 00000001800042a0     DiagnosticCommandImpl.obj
 0002:000002f0       ??_C@_0CI@LDDEGNGM@java?1lang?1UnsupportedOperationE@ 00000001800042f0     DiagnosticCommandImpl.obj
 0002:00000318       ??_C@_0DK@NFGDGGMJ@com?1sun?1management?1internal?1Dia@ 0000000180004318     DiagnosticCommandImpl.obj
 0002:00000360       ??_C@_0FA@HCGGLJHE@?$CILjava?1lang?1String?$DLLjava?1lang?1S@ 0000000180004360     DiagnosticCommandImpl.obj
 0002:000003b0       ??_C@_0BB@PPEHBGID@java?1util?1Arrays@ 00000001800043b0     DiagnosticCommandImpl.obj
 0002:000003c8       ??_C@_0CG@HHOJOFBP@?$CI?$FLLjava?1lang?1Object?$DL?$CJLjava?1util@ 00000001800043c8     DiagnosticCommandImpl.obj
 0002:000003f0       ??_C@_06ECNHPIF@asList@    00000001800043f0     DiagnosticCommandImpl.obj
 0002:000003f8       ??_C@_0BF@IEOOPILA@Invalid?5String?5Array@ 00000001800043f8     DiagnosticCommandImpl.obj
 0002:00000410       ??_C@_0DC@EEHIJFOL@com?1sun?1management?1internal?1Dia@ 0000000180004410     DiagnosticCommandImpl.obj
 0002:00000450       ??_C@_0IB@BKJILNLP@?$CILjava?1lang?1String?$DLLjava?1lang?1S@ 0000000180004450     DiagnosticCommandImpl.obj
 0002:000004d8       ??_C@_0CF@MADHDJEK@Lcom?1sun?1management?1VMOption$Or@ 00000001800044d8     Flag.obj
 0002:00000500       ??_C@_0CD@CEAHIHPC@com?1sun?1management?1VMOption$Ori@ 0000000180004500     Flag.obj
 0002:00000528       ??_C@_07MGCPDNLD@DEFAULT@  0000000180004528     Flag.obj
 0002:00000530       ??_C@_0M@BODHNBPF@VM_CREATION@ 0000000180004530     Flag.obj
 0002:00000540       ??_C@_0L@HNPILAMG@MANAGEMENT@ 0000000180004540     Flag.obj
 0002:00000550       ??_C@_0M@FDANMCLI@ENVIRON_VAR@ 0000000180004550     Flag.obj
 0002:00000560       ??_C@_0M@CEBLKBIO@CONFIG_FILE@ 0000000180004560     Flag.obj
 0002:00000570       ??_C@_09ILMJHCBE@ERGONOMIC@ 0000000180004570     Flag.obj
 0002:00000580       ??_C@_0BB@ICEJIAEF@ATTACH_ON_DEMAND@ 0000000180004580     Flag.obj
 0002:00000594       ??_C@_05NNNMIPMB@OTHER@    0000000180004594     Flag.obj
 0002:000005a0       ??_C@_0CB@NMENEKD@com?1sun?1management?1internal?1Fla@ 00000001800045a0     Flag.obj
 0002:000005d0       ??_C@_0EO@OCMOFBBM@?$CILjava?1lang?1String?$DLLjava?1lang?1O@ 00000001800045d0     Flag.obj
 0002:00000620       ??_C@_04LHKBAEFM@?$CIZ?$CJV@ 0000000180004620     Flag.obj
 0002:00000628       ??_C@_0BC@DDPBLLCP@java?1lang?1Boolean@ 0000000180004628     Flag.obj
 0002:0000063c       ??_C@_04OHLIFDMD@?$CIJ?$CJV@ 000000018000463c     Flag.obj
 0002:00000648       ??_C@_0P@MLLHBNNC@java?1lang?1Long@ 0000000180004648     Flag.obj
 0002:00000658       ??_C@_04HGHCEPA@?$CID?$CJV@ 0000000180004658     Flag.obj
 0002:00000660       ??_C@_0BB@JKEOLFJD@java?1lang?1Double@ 0000000180004660     Flag.obj
 0002:00000678       ??_C@_0CJ@FEKHENIJ@Number?5of?5Flag?5objects?5created?5@ 0000000180004678     Flag.obj
 0002:000006a8       ??_C@_0BO@EOMDLAMD@Invalid?5GarbageCollectorMBean@ 00000001800046a8     GarbageCollectorExtImpl.obj
 0002:000006c8       ??_C@_0P@CCHCOPNE@java?1lang?1Byte@ 00000001800046c8     GcInfoBuilder.obj
 0002:000006d8       ??_C@_04CCAMHLCM@?$CIB?$CJV@ 00000001800046d8     GcInfoBuilder.obj
 0002:000006e0       ??_C@_0BC@OHJKABOO@java?1lang?1Integer@ 00000001800046e0     GcInfoBuilder.obj
 0002:000006f4       ??_C@_04PFANPMCN@?$CII?$CJV@ 00000001800046f4     GcInfoBuilder.obj
 0002:00000700       ??_C@_0BA@MBLENCLH@java?1lang?1Short@ 0000000180004700     GcInfoBuilder.obj
 0002:00000710       ??_C@_04MKKJELNG@?$CIS?$CJV@ 0000000180004710     GcInfoBuilder.obj
 0002:00000718       ??_C@_0BA@HJEPPKHG@java?1lang?1Float@ 0000000180004718     GcInfoBuilder.obj
 0002:00000728       ??_C@_0BE@GKIHCGPM@java?1lang?1Character@ 0000000180004728     GcInfoBuilder.obj
 0002:0000073c       ??_C@_04JKLABMEJ@?$CIC?$CJV@ 000000018000473c     GcInfoBuilder.obj
 0002:00000748       ??_C@_0BH@KCPAAINP@Invalid?5num_attributes@ 0000000180004748     GcInfoBuilder.obj
 0002:00000760       ??_C@_0BK@KGMIKEPP@Unexpected?5num_attributes@ 0000000180004760     GcInfoBuilder.obj
 0002:00000780       ??_C@_0BG@HCNJLLGG@Invalid?5ext_att_count@ 0000000180004780     GcInfoBuilder.obj
 0002:00000798       ??_C@_0BL@CHBGEDL@Unsupported?5attribute?5type@ 0000000180004798     GcInfoBuilder.obj
 0002:000007c0       ??_C@_0IL@DNFKACMC@?$CILcom?1sun?1management?1internal?1G@ 00000001800047c0     GcInfoBuilder.obj
 0002:00000850       ??_C@_0BK@LAMMNKDJ@com?1sun?1management?1GcInfo@ 0000000180004850     GcInfoBuilder.obj
 0002:000008b8       ??_C@_06NELKLDPM@?2?$CFs?2?$CFs@ 00000001800048b8     OperatingSystemImpl.obj
 0002:000008c0       ??_C@_0L@MLLIHFJC@?2?$CFs?$CI?$CFs?$CJ?2?$CFs@ 00000001800048c0     OperatingSystemImpl.obj
 0002:000008d0       ??_C@_0O@JCGOHBMM@?2?$CFs?$CI?$CFs?$CD?$CFs?$CJ?2?$CFs@ 00000001800048d0     OperatingSystemImpl.obj
 0002:000008e0       ??_C@_0P@CIDEDEDD@PdhAddCounterA@ 00000001800048e0     OperatingSystemImpl.obj
 0002:000008f0       ??_C@_0O@HFNMDKII@PdhOpenQueryA@ 00000001800048f0     OperatingSystemImpl.obj
 0002:00000900       ??_C@_0O@EGDBAKJC@PdhCloseQuery@ 0000000180004900     OperatingSystemImpl.obj
 0002:00000910       ??_C@_0BE@GPNBOCHE@PdhCollectQueryData@ 0000000180004910     OperatingSystemImpl.obj
 0002:00000928       ??_C@_0BM@EOJADGC@PdhGetFormattedCounterValue@ 0000000180004928     OperatingSystemImpl.obj
 0002:00000948       ??_C@_0BE@BJADGCJL@PdhEnumObjectItemsA@ 0000000180004948     OperatingSystemImpl.obj
 0002:00000960       ??_C@_0BB@EBECGLNG@PdhRemoveCounter@ 0000000180004960     OperatingSystemImpl.obj
 0002:00000978       ??_C@_0BK@BKCEHIDJ@PdhLookupPerfNameByIndexA@ 0000000180004978     OperatingSystemImpl.obj
 0002:00000994       ??_C@_02DPKJAMEF@?$CFd@    0000000180004994     OperatingSystemImpl.obj
 0002:00000998       ??_C@_07OPODLDBJ@pdh?4dll@ 0000000180004998     OperatingSystemImpl.obj
 0002:000009a0       __real@3ff0000000000000    00000001800049a0     OperatingSystemImpl.obj
 0002:000009a8       __real@4059000000000000    00000001800049a8     OperatingSystemImpl.obj
 0002:000009b0       __real@bff0000000000000    00000001800049b0     OperatingSystemImpl.obj
 0002:000009b8       ??_C@_0BP@KJIDAONK@Unsupported?5Management?5version@ 00000001800049b8     management_ext.obj
 0002:000009d8       _pDefaultRawDllMain        00000001800049d8     MSVCRT:dll_dllmain.obj
 0002:000009d8       _pRawDllMain               00000001800049d8     MSVCRT:dll_dllmain.obj
 0002:000009f0       __xmm@ffffffffffffffffffffffffffffffff 00000001800049f0     MSVCRT:utility.obj
 0002:00000a00       _load_config_used          0000000180004a00     MSVCRT:loadcfg.obj
 0002:00000c00       __volatile_metadata        0000000180004c00     <linker-defined>
 0002:00000f28       __rtc_iaa                  0000000180004f28     MSVCRT:initsect.obj
 0002:00000f30       __rtc_izz                  0000000180004f30     MSVCRT:initsect.obj
 0002:00000f38       __rtc_taa                  0000000180004f38     MSVCRT:initsect.obj
 0002:00000f40       __rtc_tzz                  0000000180004f40     MSVCRT:initsect.obj
 0002:00001a8c       __IMPORT_DESCRIPTOR_jvm    0000000180005a8c     jvm:jvm.dll
 0002:00001aa0       __IMPORT_DESCRIPTOR_PSAPI  0000000180005aa0     psapi:PSAPI.DLL
 0002:00001ab4       __IMPORT_DESCRIPTOR_java   0000000180005ab4     java:java.dll
 0002:00001ac8       __IMPORT_DESCRIPTOR_KERNEL32 0000000180005ac8     kernel32:KERNEL32.dll
 0002:00001adc       __IMPORT_DESCRIPTOR_VCRUNTIME140 0000000180005adc     vcruntime:VCRUNTIME140.dll
 0002:00001af0       __IMPORT_DESCRIPTOR_api-ms-win-crt-heap-l1-1-0 0000000180005af0     ucrt:api-ms-win-crt-heap-l1-1-0.dll
 0002:00001b04       __IMPORT_DESCRIPTOR_api-ms-win-crt-stdio-l1-1-0 0000000180005b04     ucrt:api-ms-win-crt-stdio-l1-1-0.dll
 0002:00001b18       __IMPORT_DESCRIPTOR_api-ms-win-crt-string-l1-1-0 0000000180005b18     ucrt:api-ms-win-crt-string-l1-1-0.dll
 0002:00001b2c       __IMPORT_DESCRIPTOR_api-ms-win-crt-time-l1-1-0 0000000180005b2c     ucrt:api-ms-win-crt-time-l1-1-0.dll
 0002:00001b40       __IMPORT_DESCRIPTOR_api-ms-win-crt-runtime-l1-1-0 0000000180005b40     ucrt:api-ms-win-crt-runtime-l1-1-0.dll
 0002:00001b54       __IMPORT_DESCRIPTOR_api-ms-win-crt-convert-l1-1-0 0000000180005b54     ucrt:api-ms-win-crt-convert-l1-1-0.dll
 0002:00001b68       __NULL_IMPORT_DESCRIPTOR   0000000180005b68     jvm:jvm.dll
 0003:00000080       _fltused                   0000000180007080     MSVCRT:fltused.obj
 0003:00000090       __security_cookie_complement 0000000180007090     MSVCRT:gs_cookie.obj
 0003:00000098       __security_cookie          0000000180007098     MSVCRT:gs_cookie.obj
 0003:000000a0       __scrt_native_dllmain_reason 00000001800070a0     MSVCRT:utility.obj
 0003:000000a8       __isa_available            00000001800070a8     MSVCRT:cpu_disp.obj
 0003:000000ac       __isa_enabled              00000001800070ac     MSVCRT:cpu_disp.obj
 0003:000000b0       __memset_fast_string_threshold 00000001800070b0     MSVCRT:cpu_disp.obj
 0003:000000b8       __memset_nt_threshold      00000001800070b8     MSVCRT:cpu_disp.obj
 0003:000000c0       __scrt_ucrt_dll_is_in_use  00000001800070c0     MSVCRT:ucrt_stubs.obj
 0003:000001c8       jmm_interface              00000001800071c8     management_ext.obj
 0003:000001d0       jmm_version                00000001800071d0     management_ext.obj
 0003:000001d8       jvm                        00000001800071d8     management_ext.obj
 0003:00000760       ?__type_info_root_node@@3U__type_info_node@@A 0000000180007760     MSVCRT:tncleanup.obj
 0003:00000770       ?_OptionsStorage@?1??__local_stdio_scanf_options@@9@4_KA 0000000180007770     MSVCRT:default_local_stdio_options.obj
 0003:00000778       __scrt_current_native_startup_state 0000000180007778     MSVCRT:utility.obj
 0003:00000780       __scrt_native_startup_lock 0000000180007780     MSVCRT:utility.obj
 0003:000007c0       __scrt_debugger_hook_flag  00000001800077c0     MSVCRT:utility_desktop.obj
 0003:000007c4       __favor                    00000001800077c4     MSVCRT:cpu_disp.obj
 0003:000007c8       ?_OptionsStorage@?1??__local_stdio_printf_options@@9@9 00000001800077c8     <common>
 0003:000007d0       __dyn_tls_init_callback    00000001800077d0     <common>

 entry point at        0001:000024f0

 Static symbols

 0000:ffff5000       .debug$S                   0000000180000000     management_ext.exp
 0000:ffff5000       .debug$S                   0000000180000000     vcruntime:VCRUNTIME140.dll
 0000:ffff5000       .debug$S                   0000000180000000     vcruntime:VCRUNTIME140.dll
 0000:ffff5000       .debug$S                   0000000180000000     vcruntime:VCRUNTIME140.dll
 0000:ffff5000       .debug$S                   0000000180000000     vcruntime:VCRUNTIME140.dll
 0000:ffff5000       .debug$S                   0000000180000000     vcruntime:VCRUNTIME140.dll
 0000:ffff5000       .debug$S                   0000000180000000     vcruntime:VCRUNTIME140.dll
 0000:ffff5000       .debug$S                   0000000180000000     vcruntime:VCRUNTIME140.dll
 0000:ffff5000       .debug$S                   0000000180000000     ucrt:api-ms-win-crt-convert-l1-1-0.dll
 0000:ffff5000       .debug$S                   0000000180000000     ucrt:api-ms-win-crt-heap-l1-1-0.dll
 0000:ffff5000       .debug$S                   0000000180000000     ucrt:api-ms-win-crt-heap-l1-1-0.dll
 0000:ffff5000       .debug$S                   0000000180000000     ucrt:api-ms-win-crt-heap-l1-1-0.dll
 0000:ffff5000       .debug$S                   0000000180000000     ucrt:api-ms-win-crt-runtime-l1-1-0.dll
 0000:ffff5000       .debug$S                   0000000180000000     ucrt:api-ms-win-crt-runtime-l1-1-0.dll
 0000:ffff5000       .debug$S                   0000000180000000     ucrt:api-ms-win-crt-runtime-l1-1-0.dll
 0000:ffff5000       .debug$S                   0000000180000000     ucrt:api-ms-win-crt-runtime-l1-1-0.dll
 0000:ffff5000       .debug$S                   0000000180000000     ucrt:api-ms-win-crt-runtime-l1-1-0.dll
 0000:ffff5000       .debug$S                   0000000180000000     ucrt:api-ms-win-crt-runtime-l1-1-0.dll
 0000:ffff5000       .debug$S                   0000000180000000     ucrt:api-ms-win-crt-runtime-l1-1-0.dll
 0000:ffff5000       .debug$S                   0000000180000000     ucrt:api-ms-win-crt-runtime-l1-1-0.dll
 0000:ffff5000       .debug$S                   0000000180000000     ucrt:api-ms-win-crt-runtime-l1-1-0.dll
 0000:ffff5000       .debug$S                   0000000180000000     ucrt:api-ms-win-crt-runtime-l1-1-0.dll
 0000:ffff5000       .debug$S                   0000000180000000     ucrt:api-ms-win-crt-runtime-l1-1-0.dll
 0000:ffff5000       .debug$S                   0000000180000000     ucrt:api-ms-win-crt-runtime-l1-1-0.dll
 0000:ffff5000       .debug$S                   0000000180000000     ucrt:api-ms-win-crt-runtime-l1-1-0.dll
 0000:ffff5000       .debug$S                   0000000180000000     ucrt:api-ms-win-crt-runtime-l1-1-0.dll
 0000:ffff5000       .debug$S                   0000000180000000     ucrt:api-ms-win-crt-stdio-l1-1-0.dll
 0000:ffff5000       .debug$S                   0000000180000000     ucrt:api-ms-win-crt-string-l1-1-0.dll
 0000:ffff5000       .debug$S                   0000000180000000     ucrt:api-ms-win-crt-string-l1-1-0.dll
 0000:ffff5000       .debug$S                   0000000180000000     ucrt:api-ms-win-crt-time-l1-1-0.dll
 0000:ffff5000       .debug$S                   0000000180000000     kernel32:KERNEL32.dll
 0000:ffff5000       .debug$S                   0000000180000000     kernel32:KERNEL32.dll
 0000:ffff5000       .debug$S                   0000000180000000     kernel32:KERNEL32.dll
 0000:ffff5000       .debug$S                   0000000180000000     kernel32:KERNEL32.dll
 0000:ffff5000       .debug$S                   0000000180000000     kernel32:KERNEL32.dll
 0000:ffff5000       .debug$S                   0000000180000000     kernel32:KERNEL32.dll
 0000:ffff5000       .debug$S                   0000000180000000     kernel32:KERNEL32.dll
 0000:ffff5000       .debug$S                   0000000180000000     kernel32:KERNEL32.dll
 0000:ffff5000       .debug$S                   0000000180000000     kernel32:KERNEL32.dll
 0000:ffff5000       .debug$S                   0000000180000000     kernel32:KERNEL32.dll
 0000:ffff5000       .debug$S                   0000000180000000     kernel32:KERNEL32.dll
 0000:ffff5000       .debug$S                   0000000180000000     kernel32:KERNEL32.dll
 0000:ffff5000       .debug$S                   0000000180000000     kernel32:KERNEL32.dll
 0000:ffff5000       .debug$S                   0000000180000000     kernel32:KERNEL32.dll
 0000:ffff5000       .debug$S                   0000000180000000     kernel32:KERNEL32.dll
 0000:ffff5000       .debug$S                   0000000180000000     kernel32:KERNEL32.dll
 0000:ffff5000       .debug$S                   0000000180000000     kernel32:KERNEL32.dll
 0000:ffff5000       .debug$S                   0000000180000000     kernel32:KERNEL32.dll
 0000:ffff5000       .debug$S                   0000000180000000     kernel32:KERNEL32.dll
 0000:ffff5000       .debug$S                   0000000180000000     kernel32:KERNEL32.dll
 0000:ffff5000       .debug$S                   0000000180000000     kernel32:KERNEL32.dll
 0000:ffff5000       .debug$S                   0000000180000000     kernel32:KERNEL32.dll
 0000:ffff5000       .debug$S                   0000000180000000     kernel32:KERNEL32.dll
 0000:ffff5000       .debug$S                   0000000180000000     kernel32:KERNEL32.dll
 0000:ffff5000       .debug$S                   0000000180000000     kernel32:KERNEL32.dll
 0000:ffff5000       .debug$S                   0000000180000000     kernel32:KERNEL32.dll
 0000:ffff5000       .debug$S                   0000000180000000     kernel32:KERNEL32.dll
 0000:ffff5000       .debug$S                   0000000180000000     kernel32:KERNEL32.dll
 0000:ffff5000       .debug$S                   0000000180000000     psapi:PSAPI.DLL
 0000:ffff5000       .debug$S                   0000000180000000     jvm:jvm.dll
 0000:ffff5000       .debug$S                   0000000180000000     java:java.dll
 0000:ffff5000       .debug$S                   0000000180000000     java:java.dll
 0000:ffff5000       .debug$S                   0000000180000000     java:java.dll
 0000:ffff5000       .debug$S                   0000000180000000     java:java.dll
 0000:ffff5000       .debug$S                   0000000180000000     java:java.dll
 0000:ffff5000       .debug$S                   0000000180000000     java:java.dll
 0000:ffff5000       .debug$S                   0000000180000000     java:java.dll
 0001:00000adc       find_origin_constant       0000000180001adc f   Flag.obj
 0001:00001368       allocateAndInitializePdhConstants 0000000180002368 f   OperatingSystemImpl.obj
 0001:0000154c       bindPdhFunctionPointers    000000018000254c f   OperatingSystemImpl.obj
 0001:00001660       currentQueryIndexForProcess 0000000180002660 f   OperatingSystemImpl.obj
 0001:00001790       deallocateCPUCounters      0000000180002790 f   OperatingSystemImpl.obj
 0001:000018ac       getPerformanceData         00000001800028ac f   OperatingSystemImpl.obj
 0001:00001934       initializeCPUCounters      0000000180002934 f   OperatingSystemImpl.obj
 0001:00001ab4       initializeMultipleCounterForCPUs 0000000180002ab4 f   OperatingSystemImpl.obj
 0001:00001ccc       lookupNameByIndex          0000000180002ccc f   OperatingSystemImpl.obj
 0001:00001d48       makeFullCounterPath        0000000180002d48 f   OperatingSystemImpl.obj
 0001:00001e60       pdhCleanup                 0000000180002e60 f   OperatingSystemImpl.obj
 0001:00001eac       pdhInit                    0000000180002eac f   OperatingSystemImpl.obj
 0001:00001fa8       perfCPUInit                0000000180002fa8 f   OperatingSystemImpl.obj
 0001:000021a0       $$000000                   00000001800031a0     MSVCRT:amdsecgs.obj
 0001:000021d0       ?dllmain_crt_dispatch@@YAHQEAUHINSTANCE__@@KQEAX@Z 00000001800031d0 f   MSVCRT:dll_dllmain.obj
 0001:00002220       ?dllmain_crt_process_attach@@YAHQEAUHINSTANCE__@@QEAX@Z 0000000180003220 f   MSVCRT:dll_dllmain.obj
 0001:00002338       ?dllmain_crt_process_detach@@YAH_N@Z 0000000180003338 f   MSVCRT:dll_dllmain.obj
 0001:000023bc       ?dllmain_dispatch@@YAHQEAUHINSTANCE__@@KQEAX@Z 00000001800033bc f   MSVCRT:dll_dllmain.obj
 0001:00002638       capture_previous_context   0000000180003638 f   MSVCRT:gs_report.obj
 0001:00002ee0       $$000000                   0000000180003ee0     MSVCRT:guard_dispatch.obj
 0001:00002f00       $$000000                   0000000180003f00     MSVCRT:guard_xfg_dispatch.obj
 0001:00002f16       ?fin$0@?0??dllmain_crt_process_attach@@YAHQEAUHINSTANCE__@@QEAX@Z@4HA 0000000180003f16 f   MSVCRT:dll_dllmain.obj
 0001:00002f2d       ?fin$0@?0??dllmain_crt_process_detach@@YAH_N@Z@4HA 0000000180003f2d f   MSVCRT:dll_dllmain.obj
 0001:00002f46       ?fin$1@?0??dllmain_crt_process_detach@@YAH_N@Z@4HA 0000000180003f46 f   MSVCRT:dll_dllmain.obj
 0001:00002f5a       ?filt$0@?0??dllmain_dispatch@@YAHQEAUHINSTANCE__@@KQEAX@Z@4HA 0000000180003f5a f   MSVCRT:dll_dllmain.obj
 0001:00002f90       __scrt_is_nonwritable_in_current_image$filt$0 0000000180003f90 f   MSVCRT:utility.obj
 0002:00000870       MIN_UPDATE_INTERVAL        0000000180004870     OperatingSystemImpl.obj
 0002:00000874       PDH_PROCESSOR_IDX          0000000180004874     OperatingSystemImpl.obj
 0002:00000878       PDH_PROCESSOR_TIME_IDX     0000000180004878     OperatingSystemImpl.obj
 0002:0000087c       PDH_PROCESS_IDX            000000018000487c     OperatingSystemImpl.obj
 0002:00000880       PDH_ID_PROCESS_IDX         0000000180004880     OperatingSystemImpl.obj
 0002:00000888       OBJECT_COUNTER_FMT         0000000180004888     OperatingSystemImpl.obj
 0002:00000890       OBJECT_COUNTER_FMT_LEN     0000000180004890     OperatingSystemImpl.obj
 0002:00000898       OBJECT_WITH_INSTANCES_COUNTER_FMT 0000000180004898     OperatingSystemImpl.obj
 0002:000008a0       OBJECT_WITH_INSTANCES_COUNTER_FMT_LEN 00000001800048a0     OperatingSystemImpl.obj
 0002:000008a8       PROCESS_OBJECT_INSTANCE_COUNTER_FMT 00000001800048a8     OperatingSystemImpl.obj
 0002:000008b0       PROCESS_OBJECT_INSTANCE_COUNTER_FMT_LEN 00000001800048b0     OperatingSystemImpl.obj
 0002:000009e0       GS_ExceptionPointers       00000001800049e0     MSVCRT:gs_report.obj
 0002:00000f48       $unwind$Java_com_sun_management_internal_DiagnosticCommandImpl_getDiagnosticCommandInfo 0000000180004f48     DiagnosticCommandImpl.obj
 0002:00000f64       $unwind$getDiagnosticCommandArgumentInfoArray 0000000180004f64     DiagnosticCommandImpl.obj
 0002:00000f80       $unwind$Java_com_sun_management_internal_Flag_getFlags 0000000180004f80     Flag.obj
 0002:00000f9c       $unwind$Java_com_sun_management_internal_Flag_setBooleanValue 0000000180004f9c     Flag.obj
 0002:00000f9c       $unwind$Java_com_sun_management_internal_OperatingSystemImpl_getProcessCpuLoad0 0000000180004f9c     OperatingSystemImpl.obj
 0002:00000f9c       $unwind$Java_com_sun_management_internal_OperatingSystemImpl_getSystemCpuLoad0 0000000180004f9c     OperatingSystemImpl.obj
 0002:00000fa4       $unwind$Java_com_sun_management_internal_Flag_initialize 0000000180004fa4     Flag.obj
 0002:00000fa4       $unwind$bindPdhFunctionPointers 0000000180004fa4     OperatingSystemImpl.obj
 0002:00000fa4       $unwind$__raise_securityfailure 0000000180004fa4     MSVCRT:gs_report.obj
 0002:00000fa4       $unwind$__scrt_initialize_crt 0000000180004fa4     MSVCRT:utility.obj
 0002:00000fa4       $unwind$__scrt_initialize_onexit_tables 0000000180004fa4     MSVCRT:utility.obj
 0002:00000fa4       $unwind$__scrt_release_startup_lock 0000000180004fa4     MSVCRT:utility.obj
 0002:00000fa4       $unwind$__scrt_uninitialize_crt 0000000180004fa4     MSVCRT:utility.obj
 0002:00000fac       $unwind$find_origin_constant 0000000180004fac     Flag.obj
 0002:00000fb4       $unwind$Java_com_sun_management_internal_GarbageCollectorExtImpl_setNotificationEnabled 0000000180004fb4     GarbageCollectorExtImpl.obj
 0002:00000fb4       $unwind$Java_com_sun_management_internal_GcInfoBuilder_getNumGcExtAttributes 0000000180004fb4     GcInfoBuilder.obj
 0002:00000fb4       $unwind$Java_com_sun_management_internal_OperatingSystemImpl_initialize0 0000000180004fb4     OperatingSystemImpl.obj
 0002:00000fb4       $unwind$JNI_OnLoad         0000000180004fb4     management_ext.obj
 0002:00000fb4       $unwind$__scrt_initialize_default_local_stdio_options 0000000180004fb4     MSVCRT:default_local_stdio_options.obj
 0002:00000fb4       $unwind$?dllmain_crt_dispatch@@YAHQEAUHINSTANCE__@@KQEAX@Z 0000000180004fb4     MSVCRT:dll_dllmain.obj
 0002:00000fb4       $unwind$DllMain            0000000180004fb4     MSVCRT:dll_dllmain_stub.obj
 0002:00000fb4       $unwind$__GSHandlerCheck   0000000180004fb4     MSVCRT:gshandler.obj
 0002:00000fb4       $unwind$__scrt_acquire_startup_lock 0000000180004fb4     MSVCRT:utility.obj
 0002:00000fb4       $unwind$__scrt_dllmain_after_initialize_c 0000000180004fb4     MSVCRT:utility.obj
 0002:00000fb4       $unwind$__scrt_dllmain_before_initialize_c 0000000180004fb4     MSVCRT:utility.obj
 0002:00000fb4       $unwind$__scrt_dllmain_crt_thread_attach 0000000180004fb4     MSVCRT:utility.obj
 0002:00000fb4       $unwind$__scrt_dllmain_crt_thread_detach 0000000180004fb4     MSVCRT:utility.obj
 0002:00000fb4       $unwind$__scrt_dllmain_uninitialize_c 0000000180004fb4     MSVCRT:utility.obj
 0002:00000fb4       $unwind$__scrt_dllmain_uninitialize_critical 0000000180004fb4     MSVCRT:utility.obj
 0002:00000fbc       $unwind$Java_com_sun_management_internal_GcInfoBuilder_fillGcAttributeInfo 0000000180004fbc     GcInfoBuilder.obj
 0002:00000fd8       $unwind$Java_com_sun_management_internal_GcInfoBuilder_getLastGcInfo0 0000000180004fd8     GcInfoBuilder.obj
 0002:00000ff4       $unwind$_snprintf          0000000180004ff4     OperatingSystemImpl.obj
 0002:00001004       $unwind$Java_com_sun_management_internal_OperatingSystemImpl_getCommittedVirtualMemorySize0 0000000180005004     OperatingSystemImpl.obj
 0002:00001014       $unwind$Java_com_sun_management_internal_OperatingSystemImpl_getFreePhysicalMemorySize0 0000000180005014     OperatingSystemImpl.obj
 0002:00001014       $unwind$Java_com_sun_management_internal_OperatingSystemImpl_getFreeSwapSpaceSize0 0000000180005014     OperatingSystemImpl.obj
 0002:00001014       $unwind$Java_com_sun_management_internal_OperatingSystemImpl_getTotalPhysicalMemorySize0 0000000180005014     OperatingSystemImpl.obj
 0002:00001014       $unwind$Java_com_sun_management_internal_OperatingSystemImpl_getTotalSwapSpaceSize0 0000000180005014     OperatingSystemImpl.obj
 0002:00001024       $unwind$Java_com_sun_management_internal_OperatingSystemImpl_getProcessCpuTime0 0000000180005024     OperatingSystemImpl.obj
 0002:0000102c       $unwind$lookupNameByIndex  000000018000502c     OperatingSystemImpl.obj
 0002:0000102c       $unwind$pdhCleanup         000000018000502c     OperatingSystemImpl.obj
 0002:0000102c       $unwind$pdhInit            000000018000502c     OperatingSystemImpl.obj
 0002:0000102c       $unwind$perfCPUInit        000000018000502c     OperatingSystemImpl.obj
 0002:0000102c       $unwind$_RTC_Initialize    000000018000502c     MSVCRT:initsect.obj
 0002:0000102c       $unwind$_RTC_Terminate     000000018000502c     MSVCRT:initsect.obj
 0002:00001038       $unwind$makeFullCounterPath 0000000180005038     OperatingSystemImpl.obj
 0002:00001050       $unwind$currentQueryIndexForProcess 0000000180005050     OperatingSystemImpl.obj
 0002:0000106c       $unwind$initializeMultipleCounterForCPUs 000000018000506c     OperatingSystemImpl.obj
 0002:00001080       $unwind$getPerformanceData 0000000180005080     OperatingSystemImpl.obj
 0002:00001098       $unwind$allocateAndInitializePdhConstants 0000000180005098     OperatingSystemImpl.obj
 0002:000010b8       $unwind$initializeCPUCounters 00000001800050b8     OperatingSystemImpl.obj
 0002:000010dc       $unwind$deallocateCPUCounters 00000001800050dc     OperatingSystemImpl.obj
 0002:000010f0       $unwind$__GSHandlerCheckCommon 00000001800050f0     MSVCRT:gshandler.obj
 0002:000010f8       $xdatasym                  00000001800050f8     MSVCRT:amdsecgs.obj
 0002:000010fc       $unwind$?dllmain_crt_process_attach@@YAHQEAUHINSTANCE__@@QEAX@Z 00000001800050fc     MSVCRT:dll_dllmain.obj
 0002:00001138       $unwind$?fin$0@?0??dllmain_crt_process_attach@@YAHQEAUHINSTANCE__@@QEAX@Z@4HA 0000000180005138     MSVCRT:dll_dllmain.obj
 0002:00001138       $unwind$?fin$0@?0??dllmain_crt_process_detach@@YAH_N@Z@4HA 0000000180005138     MSVCRT:dll_dllmain.obj
 0002:00001138       $unwind$?fin$1@?0??dllmain_crt_process_detach@@YAH_N@Z@4HA 0000000180005138     MSVCRT:dll_dllmain.obj
 0002:00001140       $unwind$?dllmain_crt_process_detach@@YAH_N@Z 0000000180005140     MSVCRT:dll_dllmain.obj
 0002:00001194       $unwind$?dllmain_dispatch@@YAHQEAUHINSTANCE__@@KQEAX@Z 0000000180005194     MSVCRT:dll_dllmain.obj
 0002:000011bc       $unwind$?filt$0@?0??dllmain_dispatch@@YAHQEAUHINSTANCE__@@KQEAX@Z@4HA 00000001800051bc     MSVCRT:dll_dllmain.obj
 0002:000011c4       $unwind$_DllMainCRTStartup 00000001800051c4     MSVCRT:dll_dllmain.obj
 0002:000011d4       $unwind$__report_gsfailure 00000001800051d4     MSVCRT:gs_report.obj
 0002:000011dc       $unwind$capture_previous_context 00000001800051dc     MSVCRT:gs_report.obj
 0002:000011e8       $unwind$__security_init_cookie 00000001800051e8     MSVCRT:gs_support.obj
 0002:000011f4       $unwind$__scrt_is_nonwritable_in_current_image 00000001800051f4     MSVCRT:utility.obj
 0002:00001214       $unwind$__scrt_is_nonwritable_in_current_image$filt$0 0000000180005214     MSVCRT:utility.obj
 0002:0000121c       $unwind$__scrt_dllmain_exception_filter 000000018000521c     MSVCRT:utility.obj
 0002:00001230       $unwind$__scrt_fastfail    0000000180005230     MSVCRT:utility_desktop.obj
 0002:00001240       $unwind$__isa_available_init 0000000180005240     MSVCRT:cpu_disp.obj
 0002:00001250       $xdatasym                  0000000180005250     MSVCRT:guard_dispatch.obj
 0002:00001258       $xdatasym                  0000000180005258     MSVCRT:guard_xfg_dispatch.obj
 0002:00001260       .edata                     0000000180005260     management_ext.exp
 0002:00001288       rgpv                       0000000180005288     management_ext.exp
 0002:000012f4       rgszName                   00000001800052f4     management_ext.exp
 0002:00001360       rgwOrd                     0000000180005360     management_ext.exp
 0002:00001396       szName                     0000000180005396     management_ext.exp
 0002:000013a9       $N00001                    00000001800053a9     management_ext.exp
 0002:000013b4       $N00002                    00000001800053b4     management_ext.exp
 0002:00001404       $N00003                    0000000180005404     management_ext.exp
 0002:00001454       $N00004                    0000000180005454     management_ext.exp
 0002:000014a1       $N00005                    00000001800054a1     management_ext.exp
 0002:000014ef       $N00006                    00000001800054ef     management_ext.exp
 0002:00001525       $N00007                    0000000180005525     management_ext.exp
 0002:00001554       $N00008                    0000000180005554     management_ext.exp
 0002:0000158f       $N00009                    000000018000558f     management_ext.exp
 0002:000015c0       $N00010                    00000001800055c0     management_ext.exp
 0002:000015f6       $N00011                    00000001800055f6     management_ext.exp
 0002:0000162b       $N00012                    000000018000562b     management_ext.exp
 0002:0000165e       $N00013                    000000018000565e     management_ext.exp
 0002:00001693       $N00014                    0000000180005693     management_ext.exp
 0002:000016e3       $N00015                    00000001800056e3     management_ext.exp
 0002:00001726       $N00016                    0000000180005726     management_ext.exp
 0002:00001764       $N00017                    0000000180005764     management_ext.exp
 0002:000017a9       $N00018                    00000001800057a9     management_ext.exp
 0002:000017e6       $N00019                    00000001800057e6     management_ext.exp
 0002:0000183a       $N00020                    000000018000583a     management_ext.exp
 0002:0000188a       $N00021                    000000018000588a     management_ext.exp
 0002:000018d5       $N00022                    00000001800058d5     management_ext.exp
 0002:0000191d       $N00023                    000000018000591d     management_ext.exp
 0002:00001965       $N00024                    0000000180005965     management_ext.exp
 0002:000019ac       $N00025                    00000001800059ac     management_ext.exp
 0002:000019fd       $N00026                    00000001800059fd     management_ext.exp
 0002:00001a49       $N00027                    0000000180005a49     management_ext.exp
 0002:00001db4       .idata$6                   0000000180005db4     jvm:jvm.dll
 0002:00001dd4       .idata$6                   0000000180005dd4     psapi:PSAPI.DLL
 0002:00001e9c       .idata$6                   0000000180005e9c     java:java.dll
 0002:000020e8       .idata$6                   00000001800060e8     kernel32:KERNEL32.dll
 0002:00002142       .idata$6                   0000000180006142     vcruntime:VCRUNTIME140.dll
 0002:0000225e       .idata$6                   000000018000625e     ucrt:api-ms-win-crt-heap-l1-1-0.dll
 0002:0000227e       .idata$6                   000000018000627e     ucrt:api-ms-win-crt-stdio-l1-1-0.dll
 0002:0000229e       .idata$6                   000000018000629e     ucrt:api-ms-win-crt-string-l1-1-0.dll
 0002:000022c0       .idata$6                   00000001800062c0     ucrt:api-ms-win-crt-time-l1-1-0.dll
 0002:000022e0       .idata$6                   00000001800062e0     ucrt:api-ms-win-crt-runtime-l1-1-0.dll
 0002:00002302       .idata$6                   0000000180006302     ucrt:api-ms-win-crt-convert-l1-1-0.dll
 0003:00000000       ?class_name@?1??setLongValueAtObjectArray@@9@9 0000000180007000     GcInfoBuilder.obj
 0003:00000008       ?signature@?1??setLongValueAtObjectArray@@9@9 0000000180007008     GcInfoBuilder.obj
 0003:00000010       ?class_name@?1??setBooleanValueAtObjectArray@@9@9 0000000180007010     GcInfoBuilder.obj
 0003:00000018       ?signature@?1??setBooleanValueAtObjectArray@@9@9 0000000180007018     GcInfoBuilder.obj
 0003:00000020       ?class_name@?1??setByteValueAtObjectArray@@9@9 0000000180007020     GcInfoBuilder.obj
 0003:00000028       ?signature@?1??setByteValueAtObjectArray@@9@9 0000000180007028     GcInfoBuilder.obj
 0003:00000030       ?class_name@?1??setIntValueAtObjectArray@@9@9 0000000180007030     GcInfoBuilder.obj
 0003:00000038       ?signature@?1??setIntValueAtObjectArray@@9@9 0000000180007038     GcInfoBuilder.obj
 0003:00000040       ?class_name@?1??setShortValueAtObjectArray@@9@9 0000000180007040     GcInfoBuilder.obj
 0003:00000048       ?signature@?1??setShortValueAtObjectArray@@9@9 0000000180007048     GcInfoBuilder.obj
 0003:00000050       ?class_name@?1??setDoubleValueAtObjectArray@@9@9 0000000180007050     GcInfoBuilder.obj
 0003:00000058       ?signature@?1??setDoubleValueAtObjectArray@@9@9 0000000180007058     GcInfoBuilder.obj
 0003:00000060       ?class_name@?1??setFloatValueAtObjectArray@@9@9 0000000180007060     GcInfoBuilder.obj
 0003:00000068       ?signature@?1??setFloatValueAtObjectArray@@9@9 0000000180007068     GcInfoBuilder.obj
 0003:00000070       ?class_name@?1??setCharValueAtObjectArray@@9@9 0000000180007070     GcInfoBuilder.obj
 0003:00000078       ?signature@?1??setCharValueAtObjectArray@@9@9 0000000180007078     GcInfoBuilder.obj
 0003:000000d0       default_origin             00000001800070d0     Flag.obj
 0003:000000d8       vm_creation_origin         00000001800070d8     Flag.obj
 0003:000000e0       mgmt_origin                00000001800070e0     Flag.obj
 0003:000000e8       envvar_origin              00000001800070e8     Flag.obj
 0003:000000f0       config_file_origin         00000001800070f0     Flag.obj
 0003:000000f8       ergo_origin                00000001800070f8     Flag.obj
 0003:00000100       attach_origin              0000000180007100     Flag.obj
 0003:00000108       other_origin               0000000180007108     Flag.obj
 0003:00000110       main_process               0000000180007110     OperatingSystemImpl.obj
 0003:00000118       PdhAddCounter_i            0000000180007118     OperatingSystemImpl.obj
 0003:00000120       PdhOpenQuery_i             0000000180007120     OperatingSystemImpl.obj
 0003:00000128       PdhCloseQuery_i            0000000180007128     OperatingSystemImpl.obj
 0003:00000130       PdhCollectQueryData_i      0000000180007130     OperatingSystemImpl.obj
 0003:00000138       PdhGetFormattedCounterValue_i 0000000180007138     OperatingSystemImpl.obj
 0003:00000140       PdhEnumObjectItems_i       0000000180007140     OperatingSystemImpl.obj
 0003:00000148       PdhRemoveCounter_i         0000000180007148     OperatingSystemImpl.obj
 0003:00000150       PdhLookupPerfNameByIndex_i 0000000180007150     OperatingSystemImpl.obj
 0003:00000158       initializationLock         0000000180007158     OperatingSystemImpl.obj
 0003:00000188       pdhProcessImageName        0000000180007188     OperatingSystemImpl.obj
 0003:00000190       pdhIDProcessCounterFmt     0000000180007190     OperatingSystemImpl.obj
 0003:00000198       numberOfJavaProcessesAtInitialization 0000000180007198     OperatingSystemImpl.obj
 0003:0000019c       numCpus                    000000018000719c     OperatingSystemImpl.obj
 0003:000001a0       processTotalCPULoad        00000001800071a0     OperatingSystemImpl.obj
 0003:000001a8       multiCounterCPULoad        00000001800071a8     OperatingSystemImpl.obj
 0003:000001b0       cpuFactor                  00000001800071b0     OperatingSystemImpl.obj
 0003:000001b8       ?myPid@?1??getProcessID@@9@9 00000001800071b8     OperatingSystemImpl.obj
 0003:000001bc       ?initialized@?1??pdhInit@@9@9 00000001800071bc     OperatingSystemImpl.obj
 0003:000001c0       ?initialized@?1??initializePdhCPUCounters@@9@9 00000001800071c0     OperatingSystemImpl.obj
 0003:000001e0       ?__proc_attached@@3HA      00000001800071e0     MSVCRT:dll_dllmain.obj
 0003:000001f0       GS_ExceptionRecord         00000001800071f0     MSVCRT:gs_report.obj
 0003:00000290       GS_ContextRecord           0000000180007290     MSVCRT:gs_report.obj
 0003:00000788       ?is_initialized_as_dll@@3_NA 0000000180007788     MSVCRT:utility.obj
 0003:00000789       ?module_local_atexit_table_initialized@@3_NA 0000000180007789     MSVCRT:utility.obj
 0003:00000790       ?module_local_atexit_table@@3U_onexit_table_t@@A 0000000180007790     MSVCRT:utility.obj
 0003:000007a8       ?module_local_at_quick_exit_table@@3U_onexit_table_t@@A 00000001800077a8     MSVCRT:utility.obj
 0005:00000060       $R000000                   0000000180009060     management_ext.dll.res
